:020000040800F2
:10300000A810002051810008B5320008B73200082E
:10301000BB320008BF320008C332000800000000C5
:10302000000000000000000000000000C73200089F
:10303000C932000800000000CB320008CD32000881
:103040006B8100086B8100086B8100086B810008B0
:103050006B8100086B8100086B8100086B810008A0
:103060006B8100086B8100086B8100086B81000890
:103070006B8100086B8100086B8100086B81000880
:103080006B8100086B8100086B8100086B81000870
:103090006B8100086B8100086B8100086B81000860
:1030A0006B8100086B8100086B8100086B81000850
:1030B0000FAE00086B8100086B8100086B8100086F
:1030C0006B8100086B8100086B8100086B81000830
:1030D0006B810008EF7F00086B8100086B8100089E
:1030E0006B8100086B8100086B8100086B81000810
:1030F0006B8100086B8100086B8100086B81000800
:103100006B8100086B8100086B8100086B810008EF
:103110006B8100086B8100086B8100086B810008DF
:103120006B8100086B8100086B8100086B810008CF
:1031300000F002F800F06BF80AA090E8000C82445E
:103140008344AAF10107DA4501D100F060F8AFF23B
:10315000090EBAE80F0013F0010F18BFFB1A43F075
:1031600001031847C8980000E89800000A444FF08F
:10317000000C10F8013B13F0070408BF10F8014BD6
:103180001D1108BF10F8015B641E05D010F8016B1B
:10319000641E01F8016BF9D113F0080F1EBF10F87F
:1031A000014BAD1C0C1B09D16D1E58BF01F801CBA2
:1031B000FAD505E014F8016B01F8016B6D1EF9D525
:1031C0009142D6D37047000000230024002500263A
:1031D000103A28BF78C1FBD8520728BF30C148BF7A
:1031E0000B607047642908F0DF83752908F0DC83E1
:1031F000782908F01584632908F0B085732908F050
:10320000B585002070471FB51FBD10B510BD08F073
:10321000DFFD1146FFF7F7FF00F008F808F0FDFDAD
:1032200003B4FFF7F2FF03BC04F084FE002404F0B3
:1032300033FF04F011FE04F077FE4FF4E13004F0A8
:1032400087FE00F033F900F0F2FE104800681049E4
:10325000B0FBF1F0C5B20F484168284688470EA080
:1032600008F044FB10E0601C84B20A2004F030FE39
:10327000142C09D10E48006808B9012000E0002094
:103280000B4908604FF00004EDE70000000000204B
:1032900040420F007C0000200D0A20CAE4C8EB3A2F
:1032A00068656C70B2E9D1AFD6B8C1EE0D0A000006
:1032B00094812142704700BFFEE700BFFEE700BFD8
:1032C000FEE700BFFEE77047704770477047000099
:1032D0000CB50020019000906B48006840F48030ED
:1032E0006949086000BF6848006800F40030009039
:1032F0000198401C0190009818B90198B0F5A06F92
:10330000F1D16148006810F4003F02D00120009024
:1033100001E0002000900098012842D15B4800683D
:1033200040F01000594908600846006820F003008A
:1033300008600846006840F0020008605248406893
:10334000514948600846406848600846406840F473
:10335000806048600846406820F47C104860084659
:10336000406840F4E81048600846006840F080700B
:10337000086000BF4448006810F0007FFAD042485F
:10338000406820F00300404948600846406840F02B
:103390000200486000BF3C48406800F00C0008286C
:1033A000F9D10CBD10B5FFF793FF10BD10B536482D
:1033B000006840F00100344908600846406834491C
:1033C00008403149486008460068324908402E49A3
:1033D00008600846006820F48020086008464068BD
:1033E00020F4FE0048604FF41F008860FFF7DAFF0A
:1033F0004FF000602849086010BD10B50021002082
:103400000022214B5B6803F00C0121B1042906D096
:10341000082928D107E0214B214C236027E01F4BCE
:103420001F4C236023E0184B5B6803F47010164BAD
:103430005B6803F48032022303EB904022B9194BFE
:103440004343174C23600DE00F4B5B6813F4003FC0
:1034500004D0144B4343124C236003E00F4B43430F
:103460000F4C236003E00D4B0D4C236000BF00BFE9
:10347000054B5B68C3F303130B4CE15C084B1B6803
:10348000CB40074C236010BD0010024000200240DA
:103490000000FFF8FFFFF6FE08ED00E000127A00E2
:1034A0000000002000093D000400002008B50121B3
:1034B000482006F0DFF92020ADF8000010208DF83C
:1034C000030003208DF802006946094805F018FD45
:1034D0002021074805F0BFFD2020ADF80000694617
:1034E000044805F00DFD2021024805F0B4FD08BD9B
:1034F000000C014000180140FE4908807047FD495A
:10350000891C08807047FB48801C00887047F94A76
:103510001080921C1180704710B504462046FFF7BA
:10352000EBFF052004F0B1FCFFF7EDFF10BDF24802
:103530000089F04908807047EE49891C088070476F
:1035400030B5014601F01F04C1F34513CA0AE50274
:1035500005EB43151544A8B230BD00BF0100A0F132
:103560000102D0B2FAD1704710B503460C46E248CA
:103570008088A0F51341413905D0DF488088A0F547
:10358000A641103914D1DC494889FFF7B5FF18125C
:10359000FFF7B5FFD8B2FFF7B2FFD7498889FFF729
:1035A000ABFF2012FFF7ABFFE0B2FFF7A8FF5DE033
:1035B000D1488088A0F5D04104391DD1CE4880790A
:1035C000012804D1CC480088401EC01A83B2CA49E1
:1035D0004889FFF791FF1812FFF791FFD8B2FFF764
:1035E0008EFFC5498889FFF787FF2012FFF787FF05
:1035F000E0B2FFF784FF39E0BF488088A0F5AA4118
:10360000103920D1BC494889FFF776FF1812FFF71F
:1036100076FFB9494989491C88B2FFF76DFFD8B2D6
:10362000FFF76DFFB4498889FFF766FF2012FFF7A7
:1036300066FFB1498989491C88B2FFF75DFFE0B296
:10364000FFF75DFF12E0AC488079012804D1AA4859
:103650000088401EC01A83B2A74948891946FFF75F
:1036600056FFA54988892146FFF751FF10BD2DE976
:10367000F04105460E4600240027A0469E480088DB
:10368000A84203DD9C484088B04202DC0020BDE82F
:10369000F08131462846FFF767FF97488088A0F5FC
:1036A000134141390BD094488088A0F5D0410439AA
:1036B00005D091488088A0F5A641103903D12E206D
:1036C000FFF71AFF0DE08C488088A0F5AA41103959
:1036D00004D14FF43850FFF70FFF02E02220FFF72C
:1036E0000BFF85488088A0F51341203902D10220C4
:1036F000FFF733FF7F48801C008800B100240220C0
:10370000FFF72BFF7B48801C04887B488088A0F54E
:10371000134141390BD078488088A0F5A641103973
:1037200005D075488088A0F5AA4110390CD1022037
:10373000FFF713FF6F48801CB0F80080E7B24FF628
:10374000FF7000EA072708E06B488088A0F5D041A9
:10375000043902D16748801C048867488088A0F536
:103760001341253917D064488088A0F58A4135393E
:1037700011D061488088A0F58A4131390BD05E486C
:103780008088A0F50941893905D05B488088A0F57B
:103790003541053901D1204679E757488088A0F5A1
:1037A000134141390BD054488088A0F5A641103907
:1037B00005D051488088A0F5AA41103907D1E01200
:1037C000C002B91240EA411040EAE8205FE7204613
:1037D000FFF7B6FE5BE700B547488088A0F51341C8
:1037E00041390BD044488088A0F5D041043905D038
:1037F00041488088A0F5A641103903D12920FFF760
:103800007BFE0FE03C488088A0F5AA41103904D126
:103810004FF42450FFF770FE04E040F273110720CC
:10382000FFF775FE00BD00B533488088A0F5134151
:1038300041390BD030488088A0F5D041043905D0FB
:103840002D488088A0F5A641103903D12820FFF724
:1038500053FE0EE028488088A0F5AA41103904D113
:103860004FF42050FFF748FE03E000210720FFF748
:103870004EFE00BDF0B50546002400271E488079A5
:1038800001281ED11C488088A0F5D041043918D0E9
:10389000082D15D2DFE805F00406080A0C0E1012F8
:1038A00006250DE007250BE0042509E0052507E0C6
:1038B000012505E0002503E0032501E0022500BF06
:1038C00000BF0D488088A0F51341413911D00A4846
:1038D0008088A0F5D04104390BD007488088A0F536
:1038E000A641103905D004488088A0F5AA411039B6
:1038F0007ED103E0FE07006C70010020082D1CD271
:10390000DFE805F00406090C0F12151800BF14E0DB
:1039100044F0800411E044F040040EE044F0C004A0
:103920000BE044F0200408E044F0600405E044F0BB
:10393000A00402E044F0E00400BF00BFFC4880881F
:10394000A0F5AA41103902D14FF4585700E03627AC
:10395000F7488088A0F5A641103907D0F448808840
:10396000A0F5AA41103901D044F00804F04880883D
:10397000A0F5D041043901D144F002042146384673
:10398000FFF7C5FD14F0200F03D1E9488079012825
:103990000DD1E7480088E6494988884214DAE448AE
:1039A00006884088E2490880084646800CE0E048E6
:1039B0000088DF494988884206DDDD48068840885E
:1039C000DB49088008464680D9488088A0F5AA418E
:1039D000103954D1D6494889FFF78EFD0020FFF7F2
:1039E0008EFDD3494989491C88B2FFF785FD00E067
:1039F00074E00020FFF783FDCD494989891C88B216
:103A0000FFF77AFDCA490988491EC1F30F20FFF765
:103A100076FDC7494989C91C88B2FFF76DFDC449C5
:103A20000978491EC8B2FFF76AFDC1498889FFF7C6
:103A300063FD0020FFF763FDBD498989491C88B2F9
:103A4000FFF75AFD0020FFF75AFDB9498989891C03
:103A500088B2FFF751FDB6494988491EC1F30F20CE
:103A6000FFF74DFDB2498989C91C88B2FFF744FDB3
:103A7000AF498978491EC8B2FFF741FD60E0AC4903
:103A80004889FFF739FD0020FFF739FD0020FFF7D7
:103A900036FDA7490988491EC1F30F20FFF72FFD06
:103AA000A3490978491EC8B2FFF729FDA0498889B2
:103AB000FFF722FD0020FFF722FD0020FFF71FFD8A
:103AC0009B494988491EC1F30F20FFF718FD98490B
:103AD0008978491EC8B2FFF712FD31E0082D1CD2CB
:103AE000DFE805F004070A0D0F12151844F0300442
:103AF00013E044F0100410E044F020040DE000BF97
:103B00000BE044F0380408E044F0280405E044F0F9
:103B1000180402E044F0080400BF00BF8448808815
:103B2000A0F50941893904D1112746F24000044328
:103B300002E0032744F4805421463846FFF7E7FCAF
:103B4000F0BD30B504460D4629462046FFF70CFD72
:103B5000FFF7EDFC774800887749088030BD30B525
:103B600003460C46154672488088A0F5134141393A
:103B700005D06F488088A0F5A641103914D16C4952
:103B80004889FFF7B9FC1812FFF7B9FCD8B2FFF764
:103B9000B6FC67498889FFF7AFFC2012FFF7AFFC3E
:103BA000E0B2FFF7ACFC5DE061488088A0F5AA4177
:103BB000103920D15E494889FFF79EFC1812FFF7A3
:103BC0009EFC5B494989491C88B2FFF795FCD8B235
:103BD000FFF795FC56498889FFF78EFC2012FFF706
:103BE0008EFC53498989491C88B2FFF785FCE0B2F5
:103BF000FFF785FC36E04E488088A0F5D0410439B7
:103C00001DD14B488079012804D149480088401EC5
:103C1000C01A83B246494889FFF76EFC1812FFF7B5
:103C20006EFCD8B2FFF76BFC41498889FFF764FC52
:103C30002012FFF764FCE0B2FFF761FC12E03C48A1
:103C40008079012804D13A480088401EC01A83B206
:103C5000374948891946FFF75AFC35498889214672
:103C6000FFF755FC324800893349891E0880881CBB
:103C7000058030BD10B50446002C67D12C498871F1
:103C8000F02008804FF4A070488008468088A0F596
:103C9000134141390BD026488088A0F5D041043922
:103CA00005D023488088A0F5A64110391AD12C20D0
:103CB0001F4908812A2048812B2088810846808856
:103CC000A0F5D041043905D019488088A0F5A64157
:103CD000103906D14FF4A070154908804FF4F070E8
:103CE00048809CE012488088A0F50941893907D1B5
:103CF00022200F4908814E2048814F2088818EE084
:103D00000B488088A0F5AA41103917D14FF43050E4
:103D1000074908814FF4285048814FF42C5088817E
:103D20004FF4F07008804FF44870488077E00DE061
:103D300070010020140000200008006C2220FE49C1
:103D40000881202048812120888168E00120FA49EB
:103D500088714FF4A0700880F02048800846808861
:103D6000A0F51341413905D0F3488088A0F5A6415C
:103D7000103907D12C20F04908812A2048812B20B6
:103D8000888139E0EC488088A0F5D041043907D11A
:103D90002C20E94908812B2048812A2088812BE0AA
:103DA000E5488088A0F50941893907D12220E249F8
:103DB00008814F2048814E2088811DE0DE488088A0
:103DC000A0F5AA41103910D14FF43050DA490881DA
:103DD0004FF4285048814FF42C5088814FF448709C
:103DE00008804FF4F070488006E02220D249088114
:103DF0002120488120208881CF488088A0F5D041AB
:103E0000043905D0CC488088A0F5A641103906D1E8
:103E10004FF4F070C84908804FF4A070488000202B
:103E2000FFF728FD10BD2DE9FF4F04460D4616464D
:103E30001F46A019401E86B2E819401E87B2BE4830
:103E40008088A0F5134141390BD0BB488088A0F58C
:103E5000A641103905D0B8488088A0F5D041043972
:103E600020D1B5494889FFF747FB2012FFF747FBF0
:103E7000E0B2FFF744FB3012FFF741FBF0B2FFF76F
:103E80003EFBAD498889FFF737FB2812FFF737FB68
:103E9000E8B2FFF734FB3812FFF731FBF8B2FFF757
:103EA0002EFB90E0A4488088A0F5AA41103944D1A7
:103EB000A1494889FFF720FB2012FFF720FB9E490C
:103EC0004989491C88B2FFF717FBE0B2FFF717FBDF
:103ED00099494989891C88B2FFF70EFB3012FFF718
:103EE0000EFB95494989C91C88B2FFF705FBF0B262
:103EF000FFF705FB90498889FFF7FEFA2812FFF7C4
:103F0000FEFA8D498989491C88B2FFF7F5FAE8B2B3
:103F1000FFF7F5FA88498989891C88B2FFF7ECFA1E
:103F20003812FFF7ECFA84498989C91C88B2FFF777
:103F3000E3FAF8B2FFF7E3FA45E07F488079012819
:103F40000ED1A846B9467C480088801B401E80B22E
:103F5000019079480088001B401E80B2009003E069
:103F6000A046B1460195009773488088A0F50941A5
:103F700089390CD14FF0440AD34648EA09201FFA88
:103F800080F8C146452003904620029007E04FF09C
:103F9000500A4FF0510B522003905320029041469B
:103FA0005046FFF7B4FA49465846FFF7B0FA019970
:103FB0000398FFF7ACFA00990298FFF7A8FA294690
:103FC0002046FFF7D1FABDE8FF8F70B50446002602
:103FD000594805884088454357488088A0F5D04116
:103FE000043916D154488079012812D10020524951
:103FF00088712A2048812B20888100210846FFF7FC
:10400000B3FA01204C4988712B2048812A208881ED
:1040100003E000210846FFF7A7FAFFF788FA002619
:1040200002E046480480761CAE42FAD370BD00B56B
:104030009FB00121080205F010FC012140F2691037
:1040400005F018FC0120ADF8780010208DF87B00F9
:1040500003208DF87A001EA9394804F051FF4CF274
:104060003370ADF8780018208DF87B0003208DF8B0
:104070007A001EA9334804F043FF4FF68070ADF874
:10408000780018208DF87B0003208DF87A001EA997
:104090002D4804F035FF41F20100ADF878001820FA
:1040A0008DF87B0003208DF87A001EA9274804F0C4
:1040B00027FF01200890002009900F200A9000207F
:1040C0000B900C900D900E900190029003200390A5
:1040D0000020049005900690079006200F90002085
:1040E00010901190102012900020139015901490B1
:1040F000169017904FF480501890002019904FF4AC
:1041000080401A9000201B9008A81C9001A81D90C8
:104110000FA804F0D8FB0121062004F035FD322061
:1041200003F0D6FE01210020FFF7F1F9322003F061
:10413000CFFE00200CE00000700100200008006CA1
:10414000000C014000140140001801400020014013
:10415000FFF7E2F9FE49888008468088FF280ADBDD
:1041600008468088A0F57F41FF3904D0F848808850
:10417000B0F5134F7ED1D320FFF7BEF9FFF7C3F997
:10418000FFF7C1F9FFF7BFF9F14988800846808839
:104190004FF6FF7101EA0020ED498880FFF7B3F97F
:1041A000EB4989880843EA49888008468088A0F559
:1041B000134141396CD0BF20FFF79EF9FFF7A3F9F7
:1041C000FFF7A1F9FFF79FF9FFF79DF9E049888014
:1041D000084680884FF6FF7101EA0020DC4988809C
:1041E000FFF791F9DA4989880843D9498880084658
:1041F0008088A0F5D04104394AD0D420FFF77CF95B
:10420000FFF781F9FFF77FF9FFF77DF9D049888043
:10421000084680884FF6FF7101EA0020CC4988806B
:10422000FFF771F9CA4989880843C9498880084657
:104230008088A0F5A64110392AD04FF45A40FFF7E4
:104240005BF9FFF760F94FF45B40FFF755F9FFF7B3
:104250005AF9BF498880084680884FF6FF7101EA05
:104260000020BB4988804FF45C40FFF745F9FFF719
:104270004AF900E00CE0B64989880843B4498880CF
:1042800008468088B0F5004F02D145F21050888072
:10429000AF488188AFA007F029FBAD488088A0F522
:1042A000134141397ED1CF20FFF726F90020FFF7D7
:1042B00026F9C120FFF723F93020FFF720F9ED2080
:1042C000FFF71AF96420FFF71AF90320FFF717F92F
:1042D0001220FFF714F98120FFF711F9E820FFF70A
:1042E0000BF98520FFF70BF91020FFF708F97A206A
:1042F000FFF705F9CB20FFF7FFF83920FFF7FFF8AC
:104300002C20FFF7FCF80020FFF7F9F83420FFF726
:10431000F6F80220FFF7F3F8F720FFF7EDF820207A
:10432000FFF7EDF8EA20FFF7E7F80020FFF7E7F8DE
:104330000020FFF7E4F8C020FFF7DEF81B20FFF7AE
:10434000DEF8C120FFF7D8F80120FFF7D8F8C52024
:10435000FFF7D2F83020FFF7D2F83020FFF7CFF880
:10436000C720FFF7C9F8B720FFF7C9F83620FFF7D5
:10437000C3F84820FFF7C3F83A20FFF7BDF85520EF
:10438000FFF7BDF8B120FFF7B7F80020FFF7B7F847
:104390001A20FFF7B4F8B620FFF7AEF80A20FFF7AF
:1043A000AEF800E097E0A220FFF7A9F8F220FFF7AF
:1043B000A3F80020FFF7A3F82620FFF79DF80120BF
:1043C000FFF79DF8E020FFF797F80F20FFF797F829
:1043D0002A20FFF794F82820FFF791F80820FFF72C
:1043E0008EF80E20FFF78BF80820FFF788F854208E
:1043F000FFF785F8A920FFF782F84320FFF77FF841
:104400000A20FFF77CF80F20FFF779F80020FFF76C
:1044100076F80020FFF773F80020FFF770F800200F
:10442000FFF76DF8E120FFF767F80020FFF767F866
:104430001520FFF764F81720FFF761F80720FFF752
:104440005EF81120FFF75BF80620FFF758F82B20E5
:10445000FFF755F85620FFF752F83C20FFF74FF8CA
:104460000520FFF74CF81020FFF749F80F20FFF761
:1044700046F83F20FFF743F83F20FFF740F80F20B2
:10448000FFF73DF82B20FFF737F80020FFF737F84C
:104490000020FFF734F80120FFF731F83F20FFF745
:1044A0002EF82A20FFF728F80020FFF728F8002030
:1044B000FFF725F80020FFF722F8EF20FFF71FF89D
:1044C0001120FFF719F8782003F002FD2920FFF7EB
:1044D00013F803F025B91E488088A0F5D0410439AF
:1044E0007ED11120FFF708F8142003F0F1FCD02052
:1044F000FFF702F80720FFF702F84220FEF7FFFF60
:104500001D20FEF7FCFFD120FEF7F6FF0020FEF78E
:10451000F6FF1A20FEF7F3FF0920FEF7F0FFD22086
:10452000FEF7EAFF0120FEF7EAFF2220FEF7E7FF91
:10453000C020FEF7E1FF1020FEF7E1FF3B20FEF771
:10454000DEFF0020FEF7DBFF0220FEF7D8FF09E0C8
:1045500070010020204C43442049443A25780D0A3C
:10456000000000001120FEF7CAFFC520FEF7C4FFBF
:104570000320FEF7C4FFC820FEF7BEFF0020FEF7B1
:10458000BEFF2520FEF7BBFF2120FEF7B8FF052068
:10459000FEF7B5FF0020FEF7B2FF0A20FEF7AFFFDF
:1045A0006520FEF7ACFF2520FEF7A9FF7720FEF778
:1045B000A6FF5020FEF7A3FF0F20FEF7A0FF00206C
:1045C000FEF79DFFF820FEF797FF0120FEF797FF0B
:1045D000FE20FEF791FF0020FEF791FF022000E091
:1045E00035E0FEF78CFF2020FEF786FF3620FEF731
:1045F00083FF0820FEF783FF3A20FEF77DFF55205A
:10460000FEF77DFF2B20FEF777FF0020FEF777FFF8
:104610000020FEF774FF0120FEF771FF3F20FEF738
:104620006EFF2A20FEF768FF0020FEF768FF0020DB
:10463000FEF765FF0120FEF762FFDF20FEF75FFF58
:10464000782003F045FC2920FEF756FF41E7FE489D
:104650008088A0F5A641103940F07C87ED20FEF758
:104660004BFF0120FEF74BFFFE20FEF748FFEE2038
:10467000FEF742FFDE20FEF742FF2120FEF73FFF5C
:10468000F120FEF739FF0120FEF739FFDF20FEF7AA
:1046900033FF1020FEF733FFC420FEF72DFF8F20DD
:1046A000FEF72DFFC620FEF727FF0020FEF727FFAD
:1046B000E220FEF724FFE220FEF721FFE220FEF7D2
:1046C0001EFFBF20FEF718FFAA20FEF718FFB0203C
:1046D000FEF712FF0D20FEF712FF0020FEF70FFF7E
:1046E0000D20FEF70CFF0020FEF709FF1120FEF75A
:1046F00006FF0020FEF703FF1920FEF700FF002051
:10470000FEF7FDFE2120FEF7FAFE0020FEF7F7FE81
:104710002D20FEF7F4FE0020FEF7F1FE3D20FEF70F
:10472000EEFE0020FEF7EBFE5D20FEF7E8FE002027
:10473000FEF7E5FE5D20FEF7E2FE0020FEF7DFFE5D
:10474000B120FEF7D9FE8020FEF7D9FE0020FEF74B
:10475000D6FE8B20FEF7D3FE0020FEF7D0FE96207B
:10476000FEF7CDFE0020FEF7CAFEB220FEF7C4FE23
:104770000020FEF7C4FE0020FEF7C1FE0220FEF777
:10478000BEFE0020FEF7BBFE0320FEF7B8FE0020B1
:10479000FEF7B5FEB320FEF7AFFE0020FEF7AFFE3A
:1047A0000020FEF7ACFE0020FEF7A9FE0020FEF779
:1047B000A6FE0020FEF7A3FE0020FEF7A0FE0020CC
:1047C000FEF79DFE0020FEF79AFE0020FEF797FE02
:1047D0000020FEF794FE0020FEF791FE0020FEF779
:1047E0008EFE0020FEF78BFE0020FEF788FE0020E4
:1047F000FEF785FE0020FEF782FE0020FEF77FFE1A
:104800000020FEF77CFE0020FEF779FE0020FEF778
:1048100076FE0020FEF773FE0020FEF770FE0020FB
:10482000FEF76DFE0020FEF76AFEB420FEF764FE80
:104830008B20FEF764FE0020FEF761FE9620FEF757
:104840005EFE0020FEF75BFEA120FEF758FE002072
:10485000FEF755FEB520FEF74FFE0220FEF74FFE95
:104860000020FEF74CFE0320FEF749FE0020FEF775
:1048700046FE0420FEF743FE0020FEF740FEB62071
:10488000FEF73AFE0020FEF73AFE0020FEF737FE64
:10489000B720FEF731FE0020FEF731FE0020FEF7C4
:1048A0002EFE3F20FEF72BFE0020FEF728FE5E20A6
:1048B000FEF725FE0020FEF722FE6420FEF71FFE15
:1048C0000020FEF71CFE8C20FEF719FE0020FEF7EC
:1048D00016FEAC20FEF713FE0020FEF710FEDC20D3
:1048E000FEF70DFE0020FEF70AFE7020FEF707FE21
:1048F0000020FEF704FE9020FEF701FE0020FEF7E8
:10490000FEFDEB20FEF7FBFD0020FEF7F8FDDC20AE
:10491000FEF7F5FD0020FEF7F2FDB820FEF7ECFDF6
:104920000020FEF7ECFD0020FEF7E9FD0020FEF779
:10493000E6FD0020FEF7E3FD0020FEF7E0FD00208D
:10494000FEF7DDFD0020FEF7DAFD0020FEF7D7FDC3
:10495000BA20FEF7D1FD2420FEF7D1FD0020FEF79E
:10496000CEFD0020FEF7CBFD0020FEF7C8FDC120E4
:10497000FEF7C2FD2020FEF7C2FD0020FEF7BFFDBE
:104980005420FEF7BCFD0020FEF7B9FDFF20FEF726
:10499000B6FD0020FEF7B3FDC220FEF7ADFD0A20F4
:1049A000FEF7ADFD0020FEF7AAFD0420FEF7A7FDEF
:1049B0000020FEF7A4FDC320FEF79EFD3C20FEF77D
:1049C0009EFD0020FEF79BFD3A20FEF798FD00209B
:1049D000FEF795FD3920FEF792FD0020FEF78FFDD2
:1049E0003720FEF78CFD0020FEF789FD3C20FEF706
:1049F00086FD0020FEF783FD3620FEF780FD0020B7
:104A0000FEF77DFD3220FEF77AFD0020FEF777FDF0
:104A10002F20FEF774FD0020FEF771FD2C20FEF71D
:104A20006EFD0020FEF76BFD2920FEF768FD0020DB
:104A3000FEF765FD2620FEF762FD0020FEF75FFD14
:104A40002420FEF75CFD01E0700100200020FEF74D
:104A500056FD2420FEF753FD0020FEF750FD2320D5
:104A6000FEF74DFD0020FEF74AFD3C20FEF747FD16
:104A70000020FEF744FD3620FEF741FD0020FEF742
:104A80003EFD3220FEF73BFD0020FEF738FD2F20D3
:104A9000FEF735FD0020FEF732FD2C20FEF72FFD3E
:104AA0000020FEF72CFD2920FEF729FD0020FEF74F
:104AB00026FD2620FEF723FD0020FEF720FD242002
:104AC000FEF71DFD0020FEF71AFD2420FEF717FD5E
:104AD0000020FEF714FD2320FEF711FD0020FEF755
:104AE0000EFDC420FEF708FD6220FEF708FD002041
:104AF000FEF705FD0520FEF702FD0020FEF7FFFC96
:104B00008420FEF7FCFC0020FEF7F9FCF020FEF705
:104B1000F6FC0020FEF7F3FC1820FEF7F0FC002066
:104B2000FEF7EDFCA420FEF7EAFC0020FEF7E7FC10
:104B30001820FEF7E4FC0020FEF7E1FC5020FEF711
:104B4000DEFC0020FEF7DBFC0C20FEF7D8FC00208A
:104B5000FEF7D5FC1720FEF7D2FC0020FEF7CFFCB5
:104B60009520FEF7CCFC0020FEF7C9FCF320FEF7F1
:104B7000C6FC0020FEF7C3FCE620FEF7C0FC0020C8
:104B8000FEF7BDFCC520FEF7B7FC3220FEF7B7FCF0
:104B90000020FEF7B4FC4420FEF7B1FC0020FEF735
:104BA000AEFC6520FEF7ABFC0020FEF7A8FC7620EB
:104BB000FEF7A5FC0020FEF7A2FC8820FEF79FFC74
:104BC0000020FEF79CFCC620FEF796FC2020FEF796
:104BD00096FC0020FEF793FC1720FEF790FC0020C7
:104BE000FEF78DFC0120FEF78AFC0020FEF787FC13
:104BF000C720FEF781FC0020FEF781FC0020FEF7B5
:104C00007EFC0020FEF77BFC0020FEF778FCC8202D
:104C1000FEF772FC0020FEF772FC0020FEF76FFC2E
:104C20000020FEF76CFC0020FEF769FCC920FEF7AF
:104C300063FC0020FEF763FC0020FEF760FC002010
:104C4000FEF75DFC0020FEF75AFC0020FEF757FC43
:104C50000020FEF754FC0020FEF751FC0020FEF778
:104C60004EFC0020FEF74BFC0020FEF748FC002025
:104C7000FEF745FC0020FEF742FC0020FEF73FFC5B
:104C80000020FEF73CFC0020FEF739FC0020FEF778
:104C900036FCE020FEF730FC1620FEF730FC00204A
:104CA000FEF72DFC1C20FEF72AFC0020FEF727FC57
:104CB0002120FEF724FC0020FEF721FC3620FEF721
:104CC0001EFC0020FEF71BFC4620FEF718FC00200F
:104CD000FEF715FC5220FEF712FC0020FEF70FFC39
:104CE0006420FEF70CFC0020FEF709FC7A20FEF79A
:104CF00006FC0020FEF703FC8B20FEF700FC0020E2
:104D0000FEF7FDFB9920FEF7FAFB0020FEF7F7FB0C
:104D1000A820FEF7F4FB0020FEF7F1FBB920FEF718
:104D2000EEFB0020FEF7EBFBC420FEF7E8FB0020C3
:104D3000FEF7E5FBCA20FEF7E2FB0020FEF7DFFBF3
:104D4000D220FEF7DCFB0020FEF7D9FBD920FEF7CE
:104D5000D6FB0020FEF7D3FBE020FEF7D0FB0020BF
:104D6000FEF7CDFBF320FEF7CAFB0020FEF7C7FBE2
:104D7000E120FEF7C1FB1620FEF7C1FB0020FEF785
:104D8000BEFB1C20FEF7BBFB0020FEF7B8FB222079
:104D9000FEF7B5FB0020FEF7B2FB3620FEF7AFFBB7
:104DA0000020FEF7ACFB4520FEF7A9FB0020FEF734
:104DB000A6FB5220FEF7A3FB0020FEF7A0FB642019
:104DC000FEF79DFB0020FEF79AFB7A20FEF797FB8B
:104DD0000020FEF794FB8B20FEF791FB0020FEF7EE
:104DE0008EFB9920FEF78BFB0020FEF788FBA820A6
:104DF000FEF785FB0020FEF782FBB920FEF77FFB64
:104E00000020FEF77CFBC420FEF779FB0020FEF7B4
:104E100076FBCA20FEF773FB0020FEF770FBD22062
:104E2000FEF76DFB0020FEF76AFBD820FEF767FB5C
:104E30000020FEF764FBE020FEF761FB0020FEF798
:104E40005EFBF320FEF75BFB0020FEF758FBE22041
:104E5000FEF752FB0520FEF752FB0020FEF74FFB4A
:104E60000B20FEF74CFB0020FEF749FB1B20FEF752
:104E700046FB0020FEF743FB3420FEF740FB0020FA
:104E8000FEF73DFB4420FEF73AFB0020FEF737FB20
:104E90004F20FEF734FB0020FEF731FB6120FEF7C8
:104EA0002EFB0020FEF72BFB7920FEF728FB0020CD
:104EB000FEF725FB8820FEF722FB0020FEF71FFBF4
:104EC0009720FEF71CFB0020FEF719FBA620FEF73B
:104ED00016FB0020FEF713FBB720FEF710FB0020A7
:104EE000FEF70DFBC220FEF70AFB0020FEF707FBD2
:104EF000C720FEF704FB0020FEF701FBD120FEF7E0
:104F0000FEFA0020FEF7FBFAD620FEF7F8FA0020A2
:104F1000FEF7F5FADD20FEF7F2FA0020FEF7EFFAD1
:104F2000F320FEF7ECFA0020FEF7E9FAE320FEF7A3
:104F3000E3FA0520FEF7E3FA0020FEF7E0FA0A2084
:104F4000FEF7DDFA0020FEF7DAFA1C20FEF7D7FAAA
:104F50000020FEF7D4FA3320FEF7D1FA0020FEF746
:104F6000CEFA4420FEF7CBFA0020FEF7C8FA502014
:104F7000FEF7C5FA0020FEF7C2FA6220FEF7BFFA7C
:104F80000020FEF7BCFA7820FEF7B9FA0020FEF701
:104F9000B6FA8820FEF7B3FA0020FEF7B0FA9720A1
:104FA000FEF7ADFA0020FEF7AAFAA620FEF7A7FA50
:104FB0000020FEF7A4FAB720FEF7A1FA0020FEF7C2
:104FC0009EFAC220FEF79BFA0020FEF798FAC7204F
:104FD000FEF795FA0020FEF792FAD120FEF78FFA3D
:104FE0000020FEF78CFAD520FEF789FA0020FEF7A4
:104FF00086FADD20FEF783FA0020FEF780FAF32020
:10500000FEF77DFA0020FEF77AFAE420FEF774FA44
:105010000120FEF774FA0020FEF771FA0120FEF776
:105020006EFA0020FEF76BFA0220FEF768FA002005
:10503000FEF765FA2A20FEF762FA0020FEF75FFA13
:105040003C20FEF75CFA0020FEF759FA4B20FEF7F1
:1050500056FA0020FEF753FA5D20FEF750FA0020C2
:10506000FEF74DFA7420FEF74AFA0020FEF747FAE1
:105070008420FEF744FA0020FEF741FA9320FEF761
:105080003EFA0020FEF73BFAA220FEF738FA002095
:10509000FEF735FAB320FEF732FA0020FEF72FFABA
:1050A000BE20FEF72CFA0020FEF729FAC420FEF7F6
:1050B00026FA0020FEF723FACD20FEF720FA002082
:1050C000FEF71DFAD320FEF71AFA0020FEF717FAB2
:1050D000DD20FEF714FA0020FEF711FAF320FEF7A8
:1050E0000EFA0020FEF70BFAE520FEF705FA002085
:1050F000FEF705FA0020FEF702FA0020FEF7FFF99E
:105100000020FEF7FCF90220FEF7F9F90020FEF777
:10511000F6F92920FEF7F3F90020FEF7F0F93C201C
:10512000FEF7EDF90020FEF7EAF94B20FEF7E7F96C
:105130000020FEF7E4F95D20FEF7E1F90020FEF71C
:10514000DEF97420FEF7DBF90020FEF7D8F98420A1
:10515000FEF7D5F90020FEF7D2F99320FEF7CFF93C
:105160000020FEF7CCF9A220FEF7C9F90020FEF7D7
:10517000C6F9B320FEF7C3F90020FEF7C0F9BE2040
:10518000FEF7BDF90020FEF7BAF9C420FEF7B7F923
:105190000020FEF7B4F9CD20FEF7B1F90020FEF7AC
:1051A000AEF9D320FEF7ABF90020FEF7A8F9DC201A
:1051B000FEF7A5F90020FEF7A2F9F320FEF79FF90C
:1051C0000020FEF79CF9E620FEF796F91120FEF785
:1051D00096F90020FEF793F93420FEF790F90020AD
:1051E000FEF78DF95620FEF78AF90020FEF787F9C1
:1051F0007620FEF784F90020FEF781F97720FEF78C
:105200007EF90020FEF77BF96620FEF778F9002092
:10521000FEF775F98820FEF772F90020FEF76FF9A6
:105220009920FEF76CF90020FEF769F9BB20FEF724
:1052300066F90020FEF763F99920FEF760F9002077
:10524000FEF75DF96620FEF75AF90020FEF757F9E0
:105250005520FEF754F90020FEF751F95520FEF7CE
:105260004EF90020FEF74BF94520FEF748F90020E3
:10527000FEF745F94320FEF742F90020FEF73FF91B
:105280004420FEF73CF90020FEF739F9E720FEF74D
:1052900033F93220FEF733F90020FEF730F95520BC
:1052A000FEF72DF90020FEF72AF97620FEF727F900
:1052B0000020FEF724F96620FEF721F90020FEF712
:1052C0001EF96720FEF71BF90020FEF718F967208A
:1052D000FEF715F90020FEF712F98720FEF70FF907
:1052E0000020FEF70CF99920FEF709F90020FEF7DF
:1052F00006F9BB20FEF703F90020FEF700F999201C
:10530000FEF7FDF80020FEF7FAF87720FEF7F7F831
:105310000020FEF7F4F84420FEF7F1F80020FEF735
:10532000EEF85620FEF7EBF80020FEF7E8F8232011
:10533000FEF7E5F80020FEF7E2F83320FEF7DFF88D
:105340000020FEF7DCF84520FEF7D9F80020FEF734
:10535000D6F8E820FEF7D0F80020FEF7D0F80020BD
:10536000FEF7CDF89920FEF7CAF80020FEF7C7F83F
:105370008720FEF7C4F80020FEF7C1F88820FEF76A
:10538000BEF80020FEF7BBF87720FEF7B8F8002043
:10539000FEF7B5F86620FEF7B2F80020FEF7AFF88A
:1053A0008820FEF7ACF80020FEF7A9F8AA20FEF747
:1053B000A6F80020FEF7A3F8BB20FEF7A0F8002017
:1053C000FEF79DF89920FEF79AF80020FEF797F86F
:1053D0006620FEF794F80020FEF791F85520FEF7BE
:1053E0008EF80020FEF78BF85520FEF788F8002095
:1053F000FEF785F84420FEF782F80020FEF77FF8DC
:105400004420FEF77CF80020FEF779F85520FEF7DF
:1054100076F80020FEF773F8E920FEF76DF8AA2071
:10542000FEF76DF80020FEF76AF80020FEF767F837
:105430000020FEF764F80020FEF75EF8AA20FEF7D1
:105440005EF8CF20FEF758F80020FEF758F800204D
:10545000FEF755F80020FEF752F80020FEF74FF84F
:105460000020FEF74CF80020FEF749F80020FEF778
:1054700046F80020FEF743F80020FEF740F8002031
:10548000FEF73DF80020FEF73AF80020FEF737F867
:105490000020FEF734F80020FEF731F80020FEF778
:1054A0002EF80020FEF72BF80020FEF728F8F02059
:1054B000FEF722F80020FEF722F85020FEF71FF832
:1054C0000020FEF71CF80020FEF719F80020FEF778
:1054D00016F8F320FEF710F80020FEF710F8F92078
:1054E000FEF70AF80620FEF70AF81020FEF707F884
:1054F0002920FEF704F80020FEF701F83A20FDF716
:10550000FBFF5520FDF7FBFF1120FDF7F5FF6420A1
:1055100002F0DEFC2920FDF7EFFF3520FDF7ECFF60
:105520000020FDF7ECFF5120FDF7E6FFFF20FDF71F
:10553000E6FF5320FDF7E0FF2C20FDF7E0FF5520AC
:10554000FDF7DAFF8220FDF7DAFF2C20FDF7D4FF0C
:1055500002F0E6B8FE488088A0F5AA4110397DD156
:1055600055214FF47040FDF7D2FFAA214FF2010000
:10557000FDF7CDFF52214FF20200FDF7C8FF0821D1
:105580004FF20300FDF7C3FF01214FF20400FDF7C6
:10559000BEFF0D214FF43040FDF7B9FF0D214BF256
:1055A0000100FDF7B4FF0D214BF20200FDF7AFFF44
:1055B00034214FF43640FDF7AAFF34214BF201604D
:1055C000FDF7A5FF34214BF20260FDF7A0FF0D218E
:1055D0004FF43140FDF79BFF0D214BF20110FDF719
:1055E00096FF0D214BF20210FDF791FF34214FF48D
:1055F0003740FDF78CFF34214BF20170FDF787FF38
:1056000034214BF20270FDF782FF00214FF432404B
:10561000FDF77DFF00214BF20120FDF778FF00210F
:105620004BF20220FDF773FF24214FF43840FDF7C1
:105630006EFF24214BF60100FDF769FF24214BF694
:105640000200FDF764FF01214FF43F40FDF75FFFCB
:105650000F214FF43340FDF75AFF00E0FDE30F2127
:105660004BF20130FDF753FF0F214BF20230FDF7F3
:105670004EFF34214FF43940FDF749FF34214BF6FA
:105680000110FDF744FF34214BF60210FDF73FFFF8
:1056900008214FF43540FDF73AFF08214BF2015045
:1056A000FDF735FF08214BF20250FDF730FF0321D3
:1056B0004FF44240FDF72BFF24214FF43A40FDF711
:1056C00026FF24214BF60120FDF721FF24214BF674
:1056D0000220FDF71CFF00214FF43C40FDF717FFAF
:1056E00078214BF60140FDF712FF00214BF60240F6
:1056F000FDF70DFF00214FF43D40FDF708FF782135
:105700004BF60150FDF703FF00214BF60250FDF769
:10571000FEFE00214FF43E40FDF7F9FE64214BF6FA
:105720000160FDF7F4FE00214FF45140FDF7EFFE5C
:1057300033214DF20110FDF7EAFE00214DF2021077
:10574000FDF7E5FE34214DF20310FDF7E0FE0021E8
:105750004DF20410FDF7DBFE3A214DF20510FDF786
:10576000D6FE00214DF20610FDF7D1FE4A214DF282
:105770000710FDF7CCFE00214DF20810FDF7C7FE23
:105780005C214DF20910FDF7C2FE00214DF20A1016
:10579000FDF7BDFE81214DF20B10FDF7B8FE002193
:1057A0004DF20C10FDF7B3FEA6214DF20D10FDF7E2
:1057B000AEFE00214DF20E10FDF7A9FEE5214DF2DF
:1057C0000F10FDF7A4FE01214DF21010FDF79FFE12
:1057D00013214DF21110FDF79AFE01214DF2121026
:1057E000FDF795FE54214DF21310FDF790FE0121B7
:1057F0004DF21410FDF78BFE82214DF21510FDF7CE
:1058000086FE01214DF21610FDF781FECA214DF2F0
:105810001710FDF77CFE02214DF21810FDF777FE00
:1058200000214DF21910FDF772FE02214DF21A10FF
:10583000FDF76DFE01214DF21B10FDF768FE022100
:105840004DF21C10FDF763FE34214DF21D10FDF7E3
:105850005EFE02214DF21E10FDF759FE67214DF24A
:105860001F10FDF754FE02214DF22010FDF74FFEF0
:1058700084214DF22110FDF74AFE02214DF2221043
:10588000FDF745FEA4214DF22310FDF740FE022155
:105890004DF22410FDF73BFEB7214DF22510FDF728
:1058A00036FE02214DF22610FDF731FECF214DF2DA
:1058B0002710FDF72CFE02214DF22810FDF727FEE0
:1058C000DE214DF22910FDF722FE02214DF22A10B1
:1058D000FDF71DFEF2214DF22B10FDF718FE0221FF
:1058E0004DF22C10FDF713FEFE214DF22D10FDF7A9
:1058F0000EFE03214DF22E10FDF709FE10214DF290
:105900002F10FDF704FE03214DF23010FDF7FFFDCF
:1059100033214DF23110FDF7FAFD03214DF2321023
:10592000FDF7F5FD6D214DF23310FDF7F0FD00217F
:105930004FF45240FDF7EBFD33214DF20120FDF70E
:10594000E6FD00214DF20220FDF7E1FD342101E0EA
:10595000700100204DF20320FDF7D9FD00214DF22A
:105960000420FDF7D4FD3A214DF20520FDF7CFFDCF
:1059700000214DF20620FDF7CAFD4A214DF2072015
:10598000FDF7C5FD00214DF20820FDF7C0FD5C21AB
:105990004DF20920FDF7BBFD00214DF20A20FDF775
:1059A000B6FD81214DF20B20FDF7B1FD00214DF236
:1059B0000C20FDF7ACFDA6214DF20D20FDF7A7FD53
:1059C00000214DF20E20FDF7A2FDE5214DF20F2042
:1059D000FDF79DFD01214DF21020FDF798FD1321EB
:1059E0004DF21120FDF793FD01214DF21220FDF73C
:1059F0008EFD54214DF21320FDF789FD01214DF25A
:105A00001420FDF784FD82214DF21520FDF77FFD66
:105A100001214DF21620FDF77AFDCA214DF2172023
:105A2000FDF775FD02214DF21820FDF770FD0021F4
:105A30004DF21920FDF76BFD02214DF21A20FDF702
:105A400066FD01214DF21B20FDF761FD02214DF2A3
:105A50001C20FDF75CFD34214DF21D20FDF757FDA4
:105A600002214DF21E20FDF752FD67214DF21F204D
:105A7000FDF74DFD02214DF22020FDF748FD842168
:105A80004DF22120FDF743FD02214DF22220FDF7CA
:105A90003EFDA4214DF22320FDF739FD02214DF2F8
:105AA0002420FDF734FDB7214DF22520FDF72FFD11
:105AB00002214DF22620FDF72AFDCF214DF22720AD
:105AC000FDF725FD02214DF22820FDF720FDDE2106
:105AD0004DF22920FDF71BFD02214DF22A20FDF792
:105AE00016FDF2214DF22B20FDF711FD02214DF2A2
:105AF0002C20FDF70CFDFE214DF22D20FDF707FDBA
:105B000003214DF22E20FDF702FD10214DF22F2032
:105B1000FDF7FDFC03214DF23020FDF7F8FC3321A9
:105B20004DF23120FDF7F3FC03214DF23220FDF759
:105B3000EEFC6D214DF23320FDF7E9FC00214FF41E
:105B40005340FDF7E4FC33214DF20130FDF7DFFC5B
:105B500000214DF20230FDF7DAFC34214DF2033022
:105B6000FDF7D5FC00214DF20430FDF7D0FC3A21C1
:105B70004DF20530FDF7CBFC00214DF20630FDF76C
:105B8000C6FC4A214DF20730FDF7C1FC00214DF261
:105B90000830FDF7BCFC5C214DF20930FDF7B7FC85
:105BA00000214DF20A30FDF7B2FC81214DF20B309D
:105BB000FDF7ADFC00214DF20C30FDF7A8FCA6214D
:105BC0004DF20D30FDF7A3FC00214DF20E30FDF734
:105BD0009EFCE5214DF20F30FDF799FC01214DF2BD
:105BE0001030FDF794FC13214DF21130FDF78FFCBE
:105BF00001214DF21230FDF78AFC54214DF2133091
:105C0000FDF785FC01214DF21430FDF780FC822167
:105C10004DF21530FDF77BFC01214DF21630FDF7FA
:105C200076FCCA214DF21730FDF771FC02214DF2CE
:105C30001830FDF76CFC00214DF21930FDF767FCC0
:105C400002214DF21A30FDF762FC01214DF21B30AA
:105C5000FDF75DFC02214DF21C30FDF758FC3421AC
:105C60004DF21D30FDF753FC02214DF21E30FDF7C1
:105C70004EFC67214DF21F30FDF749FC02214DF229
:105C80002030FDF744FC84214DF22130FDF73FFC2C
:105C900002214DF22230FDF73AFCA4214DF22330CF
:105CA000FDF735FC02214DF22430FDF730FCB72121
:105CB0004DF22530FDF72BFC02214DF22630FDF789
:105CC00026FCCF214DF22730FDF721FC02214DF2B9
:105CD0002830FDF71CFCDE214DF22930FDF717FCC2
:105CE00002214DF22A30FDF712FCF2214DF22B3049
:105CF000FDF70DFC02214DF22C30FDF708FCFE21D2
:105D00004DF22D30FDF703FC03214DF22E30FDF74F
:105D1000FEFB10214DF22F30FDF7F9FB03214DF270
:105D20003030FDF7F4FB33214DF23130FDF7EFFB5E
:105D300003214DF23230FDF7EAFB6D214DF2333095
:105D4000FDF7E5FB00214FF45440FDF7E0FB332164
:105D50004DF20140FDF7DBFB00214DF20240FDF763
:105D6000D6FB34214DF20340FDF7D1FB00214DF26B
:105D70000440FDF7CCFB3A214DF20540FDF7C7FB8F
:105D800000214DF20640FDF7C2FB4A214DF20740CB
:105D9000FDF7BDFB00214DF20840FDF7B8FB5C218B
:105DA0004DF20940FDF7B3FB00214DF20A40FDF72B
:105DB000AEFB81214DF20B40FDF7A9FB00214DF216
:105DC0000C40FDF7A4FBA6214DF20D40FDF79FFB13
:105DD00000214DF20E40FDF79AFBE5214DF20F40F8
:105DE000FDF795FB01214DF21040FDF790FB1321CB
:105DF0004DF21140FDF78BFB01214DF21240FDF7F2
:105E000086FB54214DF21340FDF781FB01214DF239
:105E10001440FDF77CFB82214DF21540FDF777FB26
:105E200001214DF21640FDF772FBCA214DF21740D9
:105E3000FDF76DFB02214DF21840FDF768FB0021D4
:105E40004DF21940FDF763FB02214DF21A40FDF7B8
:105E50005EFB01214DF21B4000E006E3FDF757FB1E
:105E600002214DF21C40FDF752FB34214DF21D4042
:105E7000FDF74DFB02214DF21E40FDF748FB672167
:105E80004DF21F40FDF743FB02214DF22040FDF78C
:105E90003EFB84214DF22140FDF739FB02214DF2FA
:105EA0002240FDF734FBA4214DF22340FDF72FFBE8
:105EB00002214DF22440FDF72AFBB7214DF2254087
:105EC000FDF725FB02214DF22640FDF720FBCF21F7
:105ED0004DF22740FDF71BFB02214DF22840FDF754
:105EE00016FBDE214DF22940FDF711FB02214DF298
:105EF0002A40FDF70CFBF2214DF22B40FDF707FB8A
:105F000002214DF22C40FDF702FBFE214DF22D4007
:105F1000FDF7FDFA03214DF22E40FDF7F8FA1021AE
:105F20004DF22F40FDF7F3FA03214DF23040FDF71B
:105F3000EEFA33214DF23140FDF7E9FA03214DF23B
:105F40003240FDF7E4FA6D214DF23340FDF7DFFA00
:105F500000214FF45540FDF7DAFA33214DF201509C
:105F6000FDF7D5FA00214DF20250FDF7D0FA3421A9
:105F70004DF20350FDF7CBFA00214DF20450FDF72E
:105F8000C6FA3A214DF20550FDF7C1FA00214DF253
:105F90000650FDF7BCFA4A214DF20750FDF7B7FA5B
:105FA00000214DF20850FDF7B2FA5C214DF2095084
:105FB000FDF7ADFA00214DF20A50FDF7A8FA812154
:105FC0004DF20B50FDF7A3FA00214DF20C50FDF7F6
:105FD0009EFAA6214DF20D50FDF799FA00214DF2DF
:105FE0000E50FDF794FAE5214DF20F50FDF78FFAB0
:105FF00001214DF21050FDF78AFA13214DF2115094
:10600000FDF785FA01214DF21250FDF780FA542177
:106010004DF21350FDF77BFA01214DF21450FDF7BC
:1060200076FA82214DF21550FDF771FA01214DF2F9
:106030001650FDF76CFACA214DF21750FDF767FABA
:1060400002214DF21850FDF762FA00214DF219506D
:10605000FDF75DFA02214DF21A50FDF758FA0121C1
:106060004DF21B50FDF753FA02214DF21C50FDF783
:106070004EFA34214DF21D50FDF749FA02214DF23E
:106080001E50FDF744FA67214DF21F50FDF73FFA0D
:1060900002214DF22050FDF73AFA84214DF22150B1
:1060A000FDF735FA02214DF22250FDF730FAA42116
:1060B0004DF22350FDF72BFA02214DF22450FDF74B
:1060C00026FAB7214DF22550FDF721FA02214DF2B3
:1060D0002650FDF71CFACF214DF22750FDF717FA95
:1060E00002214DF22850FDF712FADE214DF229501F
:1060F000FDF70DFA02214DF22A50FDF708FAF221C0
:106100004DF22B50FDF703FA02214DF22C50FDF712
:10611000FEF9FE214DF22D50FDF7F9F903214DF264
:106120002E50FDF7F4F910214DF22F50FDF7EFF945
:1061300003214DF23050FDF7EAF933214DF2315091
:10614000FDF7E5F903214DF23250FDF7E0F96D213D
:106150004DF23350FDF7DBF900214FF45640FDF7C7
:10616000D6F933214DF20160FDF7D1F900214DF24E
:106170000260FDF7CCF934214DF20360FDF7C7F959
:1061800000214DF20460FDF7C2F93A214DF205609D
:10619000FDF7BDF900214DF20660FDF7B8F94A217F
:1061A0004DF20760FDF7B3F900214DF20860FDF7ED
:1061B000AEF95C214DF20960FDF7A9F900214DF21D
:1061C0000A60FDF7A4F981214DF20B60FDF79FF9FC
:1061D00000214DF20C60FDF79AF9A6214DF20D60F9
:1061E000FDF795F900214DF20E60FDF790F9E521DC
:1061F0004DF20F60FDF78BF901214DF21060FDF7B4
:1062000086F913214DF21160FDF781F901214DF25C
:106210001260FDF77CF954214DF21360FDF777F918
:1062200001214DF21460FDF772F982214DF21560E3
:10623000FDF76DF901214DF21660FDF768F9CA21ED
:106240004DF21760FDF763F902214DF21860FDF77A
:106250005EF900214DF21960FDF759F902214DF266
:106260001A60FDF754F901214DF21B60FDF74FF95B
:1062700002214DF21C60FDF74AF934214DF21D60F8
:10628000FDF745F902214DF21E60FDF740F9672147
:106290004DF21F60FDF73BF902214DF22060FDF742
:1062A00036F984214DF22160FDF731F902214DF2DA
:1062B0002260FDF72CF9A4214DF22360FDF727F9A8
:1062C00002214DF22460FDF722F9B7214DF225603D
:1062D000FDF71DF902214DF22660FDF718F9CF21D7
:1062E0004DF22760FDF713F902214DF22860FDF70A
:1062F0000EF9DE214DF22960FDF709F902214DF278
:106300002A60FDF704F9F2214DF22B60FDF7FFF84A
:1063100002214DF22C60FDF7FAF8FE214DF22D60BE
:10632000FDF7F5F803214DF22E60FDF7F0F810218E
:106330004DF22F60FDF7EBF803214DF23060FDF7D1
:10634000E6F833214DF23160FDF7E1F803214DF21B
:106350003260FDF7DCF86D214DF23360FDF7D7F8C0
:1063600055214FF47040FDF7D2F8AA214FF20100F9
:10637000FDF7CDF852214FF20200FDF7C8F80821D1
:106380004FF20300FDF7C3F800214FF20400FDF7C0
:10639000BEF8CC214FF43140FDF7B9F800214BF2A3
:1063A0000110FDF7B4F805214FF43640FDF7AFF8C2
:1063B00070214FF43740FDF7AAF870214BF20170BD
:1063C000FDF7A5F801214FF43840FDF7A0F80321AF
:1063D0004BF60100FDF79BF803214BF60200FDF799
:1063E00096F803214BF60300FDF791F802214FF4D4
:1063F0003C40FDF78CF800214BF60140FDF787F893
:1064000000214BF60240FDF782F8D0214FF44940BD
:10641000FDF77DF802214CF60110FDF778F85021C8
:106420004CF60210FDF773F850214CF60310FDF7FF
:106430006EF850214CF60410FDF769F800214FF476
:106440005450FDF764F855214FF46850FDF75FF89C
:106450004FF48850FDF750F8782001F016FD4FF406
:106460002450FDF749F801F05BB9FE488088A0F59B
:10647000134125397ED147F6F001E520FDF747F8B5
:106480004FF480710120FDF742F84FF4E0610220E3
:10649000FDF73DF841F230010320FDF738F8002107
:1064A0000420FDF734F840F202210820FDF72FF810
:1064B00000210920FDF72BF800210A20FDF727F81D
:1064C00000210C20FDF723F800210D20FDF71FF817
:1064D00000210F20FDF71BF800211020FDF717F811
:1064E00007211120FDF713F800211220FDF70FF806
:1064F00000211320FDF70BF800210720FDF707F816
:1065000041F290611020FDF702F840F2272111209E
:10651000FCF7FDFF9D211220FCF7F9FF4FF4C85155
:106520001320FCF7F4FF25212920FCF7F0FF0D21B3
:106530002B20FCF7ECFF07213020FCF7E8FF40F2AE
:1065400003313120FCF7E3FF03213220FCF7DFFFAA
:1065500040F206213520FCF7DAFF08213620FCF74F
:10656000D6FF40F206413720FCF7D1FF4FF44171CE
:10657000382000E057E0FCF7CAFF07213920FCF77C
:10658000C6FF40F202613C20FCF7C1FF08213D201C
:10659000FCF7BDFF00215020FCF7B9FFEF2151208F
:1065A000FCF7B5FF00215220FCF7B1FF40F23F118C
:1065B0005320FCF7ACFF4FF427416020FCF7A7FF06
:1065C00001216120FCF7A3FF00216A20FCF79FFF57
:1065D00000218020FCF79BFF00218120FCF797FF22
:1065E00000218220FCF793FF00218320FCF78FFF1E
:1065F00000218420FCF78BFF00218520FCF787FF1A
:1066000010219020FCF783FF4FF4C0619220FCF72B
:106610007EFF40F233110720FCF779FF2221002092
:10662000FCF775FF1FE78F488088A0F513412839D4
:106630007ED141F28F01EC20FCF769FF41F2342159
:10664000EF20FCF764FF4FF480710120FCF75FFF3F
:106650004FF4E0610220FCF75AFF41F230010320C1
:10666000FCF755FF00210420FCF751FF40F2022106
:106670000820FCF74CFF00210920FCF748FF00210F
:106680000A20FCF744FF01210C20FCF740FF002109
:106690000D20FCF73CFF00210F20FCF738FF002104
:1066A0001020FCF734FF07211120FCF730FF0021F8
:1066B0001220FCF72CFF00211320FCF728FF0121FA
:1066C0000720FCF724FF322001F002FC41F2904148
:1066D0001020FCF71CFF40F227211120FCF717FFC8
:1066E000322001F0F5FB8A211220FCF710FF322046
:1066F00001F0EEFB4FF4D0511320FCF708FF062108
:106700002920FCF704FF0D212B20FCF700FF32208D
:1067100001F0DEFB00212020FCF7F9FE0021212002
:10672000FCF7F5FE322001F0D3FB0021302000E021
:1067300074E0FCF7ECFE40F204613120FCF7E7FE68
:1067400040F205313220FCF7E2FE00213520FCF753
:10675000DEFE40F609413620FCF7D9FE4FF4017108
:106760003720FCF7D4FE40F201313820FCF7CFFE91
:1067700040F207713920FCF7CAFE00213C20FCF7EB
:10678000C6FE40F60A213D20FCF7C1FE322001F092
:106790009FFB00215020FCF7BAFEEF215120FCF7AF
:1067A000B6FE00215220FCF7B2FE40F23F1153200A
:1067B000FCF7ADFE4FF427416020FCF7A8FE012155
:1067C0006120FCF7A4FE00216A20FCF7A0FE002156
:1067D0008020FCF79CFE00218120FCF798FE002120
:1067E0008220FCF794FE00218320FCF790FE00211C
:1067F0008420FCF78CFE00218520FCF788FE102108
:106800009020FCF784FE4FF4C0619220FCF77FFEDD
:1068100040F233110720FCF77AFE24E61148808805
:10682000A0F5134120397DD10846FCF770FE4FF4E6
:1068300080710120FCF76BFE4FF4E0610220FCF751
:1068400066FE41F230010320FCF761FE00210420C6
:10685000FCF75DFE40F202210820FCF758FE002103
:10686000092001E070010020FCF751FE00210A2000
:10687000FCF74DFE01210C20FCF749FE00210D2004
:10688000FCF745FE00210F20FCF741FE322001F00D
:106890001FFB40F201110720FCF739FE322001F006
:1068A00017FB4FF486511020FCF731FE0721112011
:1068B000FCF72DFE4FF488711220FCF728FE4FF4F0
:1068C00030611320FCF723FE00212920FCF71FFE76
:1068D00044F210012B20FCF71AFE00215020FCF797
:1068E00016FEEF215120FCF712FE00215220FCF78A
:1068F0000EFE40F23F115320FCF709FE4FF41C51ED
:106900006020FCF704FE01216120FCF700FE00215D
:106910006A20FCF7FCFD00218020FCF7F8FD002137
:10692000812000E030E0FCF7F2FD00218220FCF73E
:10693000EEFD00218320FCF7EAFD00218420FCF716
:10694000E6FD00218520FCF7E2FD10219020FCF7F8
:10695000DEFD00219220FCF7DAFD01219320FCF7F7
:10696000D6FD4FF488719520FCF7D1FD00219720CA
:10697000FCF7CDFD00219820FCF7C9FD40F2731112
:106980000720FCF7C4FD6EE5FE488088A0F51341A2
:1069900031397DD141F21401E720FCF7B8FD4FF405
:1069A00080710120FCF7B3FD4FF400710220FCF769
:1069B000AEFD41F238010320FCF7A9FD40F20221AF
:1069C0000820FCF7A4FD00210920FCF7A0FD002110
:1069D0000A20FCF79CFD00210C20FCF798FD00210B
:1069E0000D20FCF794FD00210F20FCF790FD002105
:1069F0001020FCF78CFD07211120FCF788FD0021F9
:106A00001220FCF784FD00211320FCF780FDC82034
:106A100001F05EFA41F290611020FCF778FD40F23F
:106A200027211120FCF773FD322001F051FA0C21CF
:106A30001220FCF76CFD322001F04AFA4FF400619D
:106A40001320FCF764FD11212920FCF760FD0B21C8
:106A50002B20FCF75CFD322001F03AFA00212020C7
:106A6000FCF755FD40F23F112120FCF750FD0021BD
:106A70003020FCF74CFD4FF483713120FCF747FDCB
:106A800000213220FCF743FD4FF40171352000E076
:106A900064E0FCF73CFD41F20A613620FCF737FD6B
:106AA00040F207713720FCF732FD4FF48371382034
:106AB000FCF72DFD40F207713920FCF728FD40F26C
:106AC00002413C20FCF723FD40F60F413D20FCF73E
:106AD0001EFD00215020FCF71AFDEF215120FCF78C
:106AE00016FD00215220FCF712FD40F23F11532009
:106AF000FCF70DFD4FF41C516020FCF708FD01214F
:106B00006120FCF704FD00216A20FCF700FD002154
:106B10008020FCF7FCFC00218120FCF7F8FC002120
:106B20008220FCF7F4FC00218320FCF7F0FC00211C
:106B30008420FCF7ECFC00218520FCF7E8FC102108
:106B40009020FCF7E4FC4FF4C0619220FCF7DFFCDE
:106B500040F233110720FCF7DAFC84E4894880888E
:106B6000A0F5A84108397DD14FF480710120FCF7D0
:106B7000CEFC4FF4E0610220FCF7C9FC41F2300189
:106B80000320FCF7C4FC00210420FCF7C0FC40F209
:106B900007210820FCF7BBFC00210920FCF7B7FC0B
:106BA00000210A20FCF7B3FC00210C20FCF7AFFC0D
:106BB00000210D20FCF7ABFC00210F20FCF7A7FC07
:106BC000142001F085F941F2B0611020FCF79FFC20
:106BD00001211120FCF79BFC01211720FCF797FCF9
:106BE0004FF49C711220FCF792FC4FF400611320CB
:106BF000FCF78DFC09212920FCF789FC09212A20BA
:106C0000FCF785FC0021A420FCF781FC002150202A
:106C1000FCF77DFCEF215120FCF779FC002152208C
:106C2000FCF775FC40F23F115320FCF770FC4FF469
:106C30001C516020FCF76BFC01216120FCF767FC14
:106C400000216A20FCF763FC00218020FCF75FFC38
:106C500000218120FCF75BFC00218220FCF757FC1F
:106C6000002100E024E08320FCF751FC0021842077
:106C7000FCF74DFC00218520FCF749FC13219020F6
:106C8000FCF745FC00219220FCF741FC03219320F6
:106C9000FCF73DFC4FF488719520FCF738FC40F27E
:106CA00073110720FCF733FC322001F011F9B9E42D
:106CB00034488088A0F5A851053965D10720FCF734
:106CC00026FC322001F004F94FF48E711220FCF7FB
:106CD0001EFC0121A420FCF71AFC0F210820FCF760
:106CE00016FC08210A20FCF712FC08210D20FCF7F5
:106CF0000EFC40F207713020FCF709FC072131201F
:106D0000FCF705FC40F203613220FCF700FC4FF475
:106D1000E0613320FCF7FBFB40F202213420FCF75A
:106D2000F6FB02213520FCF7F2FB41F60F7136200D
:106D3000FCF7EDFB40F207713720FCF7E8FB002180
:106D40003820FCF7E4FB00213920FCF7E0FB40F29F
:106D500007713A20FCF7DBFB00213B20FCF7D7FB57
:106D600007213C20FCF7D3FB00213D20FCF7CFFBA3
:106D7000322001F0ADF801210720FCF7C8FB01210A
:106D8000172002E070010020AEE0FCF7C0FB3220CB
:106D900001F09EF84FF4BD511020FCF7B8FB40F213
:106DA00017211120FCF7B3FB4FF48F711220FCF771
:106DB000AEFB4FF470611320FCF7A9FB00212A20E1
:106DC000FCF7A5FB0A212920FCF7A1FB4FF49F71DA
:106DD0001220FCF79CFB00215020FCF798FBEF21D0
:106DE0005120FCF794FB00215220FCF790FB40F26D
:106DF0003F115320FCF78BFB4FF41C516020FCF734
:106E000086FB01216120FCF782FB00216A20FCF750
:106E10007EFB00218020FCF77AFB00218120FCF71B
:106E200076FB00218220FCF772FB00218320FCF717
:106E30006EFB00218420FCF76AFB00218520FCF713
:106E400066FB13219020FCF762FB4FF44071922007
:106E5000FCF75DFB05219320FCF759FB00219520F1
:106E6000FCF755FB00219720FCF751FB00219820EF
